:100054000000000000006301630173000800FF005A
:1000640000005300090050000C0033000900500048
:100074000C001300090050000C00190013001100BB
:100084000700090003000100010000007B52433512
:1000940033312D48462052464944205265616465F7
:1000A40072204669726D776172652056312E337DF8
:1000B400003030303030303030303030303030306C
:1000C4003000002401E00EBF03EE0DBFD2E0C4E611
:1000D400B0E0A0E6F0E0E4E590E082E715901D9240
:1000E4000197E1F7B0E0A2ED90E082EF0D92019765
:1000F400E9F70C94790E602D10C0E199FECF472FDB
:10010400582F460F501D5FBB4EBBFD01E60FF01D7F
:1001140050815DBBE29AE19A6F5F691770F30895AD
:10012400E199FECF602D0DC0472F582F460F501D6B
:100134005FBB4EBBE09A5DB3FD01E60FF01D50833B
:100144006F5F691788F308953A932A931A932B2FB4
:100154001A2FC498B22FBB0FBE773B2FB32F0E9428
:10016400D416B12F0E94D416C49A199129913991A9
:1001740008953A932A931A931B2FC498B12FBB0F57
:10018400BE773B2F3068B32F0E94D416B02D0E9447
:10019400D416BFB12B2FC49AB22F1991299139913A
:1001A40008953A932A931A932B2F1A2FA22FBB2721
:1001B40088E0902D0E941A173A2FB02DA32FC4DF88
:1001C400B22FA12FC1DF19912991399108953A9342
:1001D4002A931A931B2FA12FBB2788E0902D0E94EE
:1001E4001A173A2FB02DA32FAFDFB12FC2DF2B2F59
:1001F400B22F19912991399108953A932A931A9318
:100204000A93FA92EA92DA92CA92BA92AA929A92C9
:100214008A927A926A925A92BB2E792E8A2E572EFD
:10022400682EE52EF62E102DBFE1DB2EC02C302DCE
:10023400202DB2E00B2FB6E0AFE7B3DFB7E0AFE7B6
:10024400B0DF0E94140EB5E0C2DFB6FFFCCFB1E010
:10025400A02DA7DFB9E2BBDF9B2EB9E2A0E2A1DFAC
:10026400E0926000F09261007092620080926300FC
:100274005092640060926500F7010486BBB7B062D7
:10028400BBBFFB2DF030D1F0F130D9F0F33009F1E0
:10029400F73079F1FB3029F1FC3089F1F231A1F129
:1002A400F431C1F1F631D9F1F93109F455C0FA311B
:1002B40009F458C0FE3109F45BC075C0302D202DFF
:1002C40074C0002DB1E13B2FB0E12B2FF7EFDF22FB
:1002D4006CC0002DB7E03B2FB4E02B2FF7EFDF22EB
:1002E40064C0002DF7EFDF22B5E03B2FB4E02B2FE5
:1002F4005CC0002DB5E03B2FB4E02B2F56C0B5E019
:100304003B2FB4E02B2F51C0002DB1E13B2FB0E1C6
:100314002B2F4BC0B4E03B2FB4E02B2F46C0BFE0E3
:1003240056DFAB2FBB2794E0B595A7959A95E1F7D7
:10033400B095A195BF4FCD01AA2797FDA095BA2FDF
:10034400F70180879187A287B387B4E00B2FB6E0CB
:100354003B2FB4E02B2F29C0002DB5E03B2FB4E098
:100364002B2F23C0002DB5E03B2FB4E02B2F1DC055
:10037400BFE02DDFAB2FBB2794E0B595A7959A95E9
:10038400E1F7B095A195BF4FCD01AA2797FDA095A0
:10039400BA2FF70180879187A287B387BDE33B2FEC
:1003A400B4E02B2F02C0B9E11B2F101509F0E1C0F6
:1003B400BAE10DDFB074CB2EC01421F4BAE1A0E48D
:1003C4000E94180E30622062B6E0A32FA068E9DE16
:1003D400BBE2A02FE6DE01FD04C0B9E0A2E00E946A
:1003E400180EB1E0AB2DDDDEB22FE0916000F0918C
:1003F4006100A485BA23B015B9F3B9E0A4E00E9462
:10040400180EB6E0AFE7CDDEB7E0AFE7CADEB1E085
:10041400A02DC7DEE0916000F0916100B1811B2F37
:10042400E0916000F0916100B485B5FF0DC0E091EA
:100434006000F0916100B785E0916000F091610087
:100444003E96A081AB2BA083E0916000F091610007
:100454003E96B081BD21B083E0916000F0916100CF
:10046400B685B015D9F1E0916000F0916100B685D0
:10047400B0FF07C0BBE0ABDEF701B587BAE11B2FC5
:1004840009C0E0916000F0916100B685B1FF02C03F
:10049400B8E01B2FE0916000F0916100B685B2FFD7
:1004A40003C0B7E11B2F1AC0E0916000F091610016
:1004B400B685B4FF05C00E94140EB5E11B2F0EC013
:1004C400E0916000F0916100B685B3FF03C0B4E031
:1004D4001B2F04C0101511F4B4E61B2FFEE1BF1648
:1004E40019F0F6E1BF16F9F5B5E071DEB770AB2E81
:1004F400A014F9F0F701A681B781AA0FBB1FAA0FB8
:10050400BB1FAA0FBB1FAA0DB01DA850B009CD0177
:10051400AA27BB27F70138964081518162817381F4
:10052400480F591F6A1F7B1F408351836283738363
:100534001AC0F701A681B781AA0FBB1FAA0FBB1F60
:10054400AA0FBB1FCD01AA27BB27F701389640810C
:10055400518162817381480F591F6A1F7B1F408339
:10056400518362837383C01421F4BAE1A0E40E942E
:100574002B0EBBB7BF7DBBBF009260000092610031
:100584000092620000926300009264000092650091
:10059400B9E2A92D06DEB12F59906990799089901E
:1005A4009990A990B990C990D990E990F99009913E
:1005B4001991299139910895FA93EA93BA93AA93D8
:1005C4009A938A937A936A935A934A933A931A9290
:1005D4000A921FB61A920024A0916000B0916100A3
:1005E400109709F483C1A0916200B0916300109741
:1005F40009F47CC1A0916400B0916500109709F4DE
:1006040075C1B02DB6DDB093D400BAE0E0DDBF70A3
:10061400E0916000F0916100B68760C1B6E0D7DD7B
:10062400B093D300B7E0D3DDA091D300BA23B09345
:10063400D200B091D200E0916000F09161003C964C
:10064400A081AB2BA083B091D200B0FF57C0B0E41F
:100654003B2FB4E0BCDD3B1B3093D500A091D5000B
:10066400BB27E0916000F091610084819581E09165
:100674006000F091610062817381861B970BA8175B
:10068400B90780F0E0916000F0916100B481E091DD
:100694006000F0916100A281BA1BB093D500B6E06E
:1006A400A1E07FDD0092D60020C0B2E0E0916000BE
:1006B400F09161009281A381E0916200F091630066
:1006C4009E0FAF1FE92FFA2FA0816BDDE091600030
:1006D400F09161003296A081B1811196A083B1831B
:1006E400B091D600BF5FB093D600B091D600A09170
:1006F400D500BA17D0F2B7E0A1E053DDB091D20033
:10070400B4FF13C0B7E0A0E14CDDB6E0A2E849DDD8
:10071400E0916000F0916100B089B01531F0B2E26F
:10072400A2E03FDDB02DA02D0FDDB091D200B3FFCC
:1007340037C0E0916000F0916100B189B01539F4DF
:10074400E0916000F0916100B685B01549F4B1E024
:10075400A02D27DDB091D200B460B093D20020C0A8
:10076400E0916000F0916100B685E0916000F09145
:100774006100B787E0916000F09161000686B9E0FE
:10078400A1E00FDDE0916000F09161000682078234
:10079400B091D200B77FB093D200B7E0A8E001DDFA
:1007A400B091D200BE70B01509F453C0B4E00FDDAF
:1007B400B093D5000092D60031C0E0916000F09172
:1007C4006100A681B781A034B005E0F4B2E0FFDC9B
:1007D400E0916000F09161009681A781E09164004E
:1007E400F09165009E0FAF1FE92FFA2FB083E091BF
:1007F4006000F09161003696A081B1811196A083CA
:10080400B18307C0B0E7E0916000F0916100B1836B
:100814000BC0B091D600BF5FB093D600B091D600A4
:10082400A091D500BA1748F2B4E0D1DCB093D5005A
:10083400E0916000F0916100B181B01529F4B091AC
:10084400D500B01509F0B6CFB7E0A091D200AA70D8
:10085400A8DCB091D200B1FF0EC0B3E0B8DCB07731
:10086400B03749F4B9E0B3DCB093D600B9E0A09155
:10087400D600A46096DCB091D200B2FF1BC0B6E0F3
:10088400A0E28FDCB7E0A4E28CDCB091D200BF7DA3
:10089400B093D200E0916000F09161003C96B08189
:1008A400BF7DB083E0916000F09161003C96B0811F
:1008B400B460B083B091D200B5FF10C0B7E0A0E23D
:1008C40070DCE0916000F0916100B181B01531F409
:1008D400B1E0E0916000F0916100B183B3E077DCB6
:1008E400B3FD9CCEB02DA091D4005BDC19901FBE4B
:1008F4000990199039914991599169917991899106
:100904009991A991B991E991F99118953A932A93FA
:100914001A930A930B2F192F2A2F302D0E94A80DFA
:100924003B2FB01509F092C08CE3902DA02DB02D73
:100934000E94F40CB2E2A3E034DCB9E0A8E00E9427
:100944002B0EBFE0A7E02DDC0092A8010092A901C4
:100954000092B4010092AA010092AB010092AC0192
:100964000092AD010092AE010092AF01E0EBF1E024
:1009740000820182028203820092B5010092B601D4
:100984000092B7010092B8010092B901E0916600AB
:10099400F09167000083A1E0BB27A093AC01B09362
:1009A400AD01B1E0B093B901BEE190916600A091B0
:1009B4006700709168008091690058EA61E01DDC6D
:1009C4003B2F301569F4E0EBF1E080819181A28145
:1009D400B38180319005A005B00511F0BDE03B2F37
:1009E4003A3161F4E0EBF1E080819181A281B3813D
:1009F40080319005A005B00509F4302DA091AE0119
:100A0400B091AF01A230B00558F0B22FA12F809160
:100A140068009091690062E0702D0E94521716C020
:100A2400A091AE01B091AF01A130B00549F4E091BD
:100A34006800F0916900B081E12FF22FB08303C008
:100A4400E12FF22F0082E12FF22F0182B32F0991BF
:100A540019912991399108953A932A931A933B2F26
:100A6400192F2A2FB3E9A32F922F812F04D0199184
:100A74002991399108953A932A931A930A93FA92F1
:100A8400EA92DA92CA92BA92AA929A928A927A9242
:100A94006A925A924A923A9224977B2EEA2E582EC0
:100AA400692E102DF02C002DD02C202D302DC02C93
:100AB400A02C902CB02C802C0E94A80D1B2FB015BC
:100AC40009F0A4C18AE6902DA02DB02D8BD7DE01AC
:100AD400962D852D64E0702D0E945217BAE1A8E28C
:100AE40060DBB9E0A8E00E942B0ED02C8AC1F1E2B1
:100AF400EF1618F0BCE31B2F84C10092A8010092EA
:100B0400A9010092B4010092AA010092AB010092E3
:100B1400AC010092AD010092AE010092AF01E0EB96
:100B2400F1E000820182028203820092B501009208
:100B3400B6010092B7010092B8010092B901709217
:100B4400A801B1E0B093B901B2E2A3E02ADBAE2D73
:100B5400BB2788E0902D0E942D170A2F001521F144
:100B6400BFE0A02F902F990F990F990F990FA92BE0
:100B740018DBAE2DBB2788E0902D0E941A17AF5FBB
:100B8400FA2E0730C1F4B1E0B093B80187E0992799
:100B9400AA27BB27E0EBF1E080839183A283B38390
:100BA400BFE0A02FFEDA07C0AE2DBB2788E0902D52
:100BB4000E941A17FA2EE0916600F0916700708285
:100BC400AE2DBB2788E0902D0E941A17AA0FAA0FFA
:100BD400AA0FAA0FA05EA00FE0916600F091670033
:100BE400A183202D302D0EC0FE01E20FF31FB08132
:100BF400F90190916600A0916700E90FFA1FB28392
:100C04002F5F3F4FAF2DBB272A173B076CF3AF2D48
:100C1400BB271296A093AC01B093AD01BEE19091B5
:100C24006600A0916700709168008091690058EA9D
:100C340061E0E3DA1B2FB091B801B01509F464C088
:100C4400B02C202D302D2CC0F901A0916800B0915A
:100C54006900EA0FFB1FB0818B2EF901A091680097
:100C6400B0916900EA0FFB1FB081A7E0A21BAA2381
:100C740019F0BB0FAA95E9F7AB2D922F9F5F99232B
:100C840019F0A6959A95E9F7BA2BF90190916800A5
:100C9400A0916900E90FFA1FB083B82C2F5F3F4F72
:100CA400A091AE01B091AF012A173B0768F2E0EBC7
:100CB400F1E080819181A281B3814091AE01509194
:100CC400AF0166277727841B950BA60BB70B809380
:100CD400B0019093B101A093B201B093B301B0916C
:100CE400B501B01589F0B091B501A7E04A2E3B2EAD
:100CF400A091B501BB27169689E0902D0E941A1782
:100D04004A1A340C3092B501101519F01A3109F051
:100D140078C0C02C088209820A820B82001591F0E7
:100D2400E0916800F0916900B081FE013197EF0D08
:100D3400F01DA081BA2BFE013197EF0DF01DB08399
:100D4400B1E0CB2E202D302D14C0F901EC0DF01D97
:100D5400A0916800B0916900EA0FFB1FB081F9010E
:100D6400EF0DF01D9C2FAD2FE90FFA1FB0832F5FFD
:100D74003F4FA4E0BB278F2D9927A81BB90B2A1737
:100D84003B071CF3E0EBF1E080819181A281B38108
:100D940068E277274E2D5527641B750BAB01662738
:100DA40057FD6095762F84179507A607B70719F0A6
:100DB400BDE01B2F26C01A31F1F0B981A881BA27F2
:100DC400AA81BA27AB81BA27AB2EE091AE01F0918C
:100DD400AF01A0916800B0916900EA0FFB1FE150D8
:100DE400F009B0819B2EA91419F0BAE01B2F09C099
:100DF400B1E0DB2E06C0B091B501BE0DB01BEB2EE9
:100E0400102DD01419F4101509F471CEB62DA52D9A
:100E1400CE0164E0702D0E945217BAE1A0E219D706
:100E2400B12F24963990499059906990799089907E
:100E34009990A990B990C990D990E990F9900991A5
:100E440019912991399108953A932A931A930A93FF
:100E54009D018C01B3E9A32F922F812F702F05D010
:100E6400099119912991399108953A932A931A93E2
:100E74000A93FA92EA92EB2E192F2A2FF72E082FB3
:100E8400302D64D63B2FB01509F098C08AE6902D1A
:100E9400A02DB02DA7D5B2E2AFE083D9B9E0A8E088
:100EA400D8D60092A8010092A9010092B401009240
:100EB400AA010092AB010092AC010092AD01009234
:100EC400AE010092AF01E0EBF1E000820182028208
:100ED40003820092B5010092B6010092B70100921C
:100EE400B8010092B901E0916600F0916700E082D8
:100EF400B0E7E0916600F0916700B183A0916600CD
:100F0400B09167001296922F812F64E0702D0E9499
:100F14005217E0916600F0916700B381E09166009A
:100F2400F0916700A281BA27E0916600F091670012
:100F3400A481BA27E0916600F0916700A581BA27E1
:100F4400E0916600F0916700B683A7E0BB27A09309
:100F5400AC01B093AD01B1E0B093B901BEE19091A1
:100F64006600A0916700709168008091690058EA5A
:100F740061E043D93B2FEF2DF02F00823015B1F4FF
:100F8400E0EBF1E080819181A281B381883090050A
:100F9400A005B00519F0BDE03B2F08C0A3EAB1E0FD
:100FA400922F812F64E0702D0E945217E091680007
:100FB400F0916900B081EF2DF02FB083B32FE99049
:100FC400F990099119912991399108953A932A93A5
:100FD4001A933B2F192F2A2FB0E3A32F90E1822FCE
:100FE400712F04D019912991399108953A932A9334
:100FF4001A930A93FA92EA92DA92CA92BA92CB2E8E
:10100400BA2E292FF72E082F302DD02C0BD680E89E
:1010140092E0A02DB02DE6D4B2E2AFE0C2D80092A7
:10102400A8010092A9010092B4010092AA010092C1
:10103400AB010092AC010092AD010092AE010092AE
:10104400AF01E0EBF1E000820182028203820092B0
:10105400B5010092B6010092B7010092B801009266
:10106400B901E0916600F0916700C082E0916600EA
:10107400F0916700B182A2E0BB27A093AC01B093CA
:10108400AD01BEE190916600A09167007091680087
:101094008091690058EA61E0B0D83B2F301509F41B
:1010A4008BC0313009F47FC0E0EBF1E080819181A5
:1010B400A281B38188309005A005B00509F5BAE195
:1010C40086D8B0FF1DC0E0916800F0916900A0814E
:1010D400BB27AF70B02DE0916800F091690090815A
:1010E40092959F70892F99278F70902DA817B90713
:1010F40019F4B8E0EB2E06C0B1E23B2FE02C02C09D
:10110400B4E0EB2EE0EBF1E080819181A281B38128
:101114004E2D55276627772784179507A607B70707
:10112400A9F4E0916800F0916900B081BF70B083C8
:10113400E0916800F0916900B081BA70B01519F4BB
:10114400BCE03B2F7BC0B9E03B2F78C0A091AE013F
:10115400B091AF01822F9927A817B90758F0B02F83
:10116400AF2D8091680090916900622F77270E94CB
:10117400521764C0B02FAF2D809168009091690020
:101184006091AE017091AF010E945217B091AE010F
:101194001B2F06C0F02FEF2DE10FF01D00821F5F03
:1011A4001217C0F34BC0B02FAF2D81EC90E0622F2B
:1011B40077270E94521742C0A091AE01B091AF01AF
:1011C400822F9927A817B90779F1BEE03B2FA09188
:1011D400AE01B091AF01822F9927A817B90758F033
:1011E400B02FAF2D8091680090916900622F77270E
:1011F4000E94521723C0B02FAF2D809168009091A8
:1012040069006091AE017091AF010E945217B091D4
:10121400AE011B2F06C0F02FEF2DE10FF01D008251
:101224001F5F1217C0F30AC0B02FAF2D8091680062
:1012340090916900622F77270E945217B32FB990BB
:10124400C990D990E990F99009911991299139910E
:1012540008953A932A931A933B2F192F2A2FB0EA11
:10126400A32F90E1822F712F04D0199129913991E4
:1012740008953A932A931A930A93FA92EA92DA9285
:101284000B2FFA2E192FD72EE82E302D80ED97E054
:10129400A02DB02DA7D3B2E2A7E00E94D300009204
:1012A400A8010092A9010092B4010092AA0100923F
:1012B400AB010092AC010092AD010092AE0100922C
:1012C400AF01E0EBF1E0008201820282038200922E
:1012D400B5010092B6010092B7010092B8010092E4
:1012E400B901E0916600F09167000083E091660027
:1012F400F0916700F182A2E0BB27A093AC01B09308
:10130400AD01BEE190916600A09167007091680004
:101314008091690058EA61E00E94FF003B2F313060
:1013240009F46AC0E0EBF1E080819181A281B3818C
:1013340088309005A005B00501F5BAE10E94E900E6
:10134400B0FF1BC0E0916800F0916900A081BB2749
:10135400AF70B02DE0916800F09169009081929592
:101364009F70892F99278F70902DA817B90719F4AA
:10137400B8E02B2F04C0202D02C0B4E02B2FE0EBEB
:10138400F1E080819181A281B381422F55276627A4
:10139400772784179507A607B707A9F4E091680093
:1013A400F0916900B081BF70B083E0916800F09162
:1013B4006900B081BA70B01519F4BCE03B2F1CC0B1
:1013C400B9E03B2F19C0E0916800F0916900B08149
:1013D400BF70B083E0916800F0916900B081FB2F89
:1013E400F03019F0FA3021F005C0BCE03B2F04C006
:1013F400302D02C0B9E03B2F301509F0ABC000928C
:10140400A8010092A9010092B4010092AA010092DD
:10141400AB010092AC010092AD010092AE010092CA
:10142400AF01E0EBF1E000820182028203820092CC
:10143400B5010092B6010092B7010092B801009282
:10144400B901A0916600B09167009E2D8D2D612F8A
:1014540077270E9452171093AC010092AD01BEE1B0
:1014640090916600A0916700709168008091690076
:1014740058EA61E00E94FF003B2F313009F46AC052
:10148400E0EBF1E080819181A281B3818830900505
:10149400A005B00501F5BAE10E94E900B0FF1BC048
:1014A400E0916800F0916900A081BB27AF70B02D76
:1014B400E0916800F0916900908192959F70892F66
:1014C40099278F70902DA817B90719F4B8E02B2F1E
:1014D40004C0202D02C0B4E02B2FE0EBF1E08081AA
:1014E4009181A281B381422F5527662777278417DC
:1014F4009507A607B707A9F4E0916800F091690081
:10150400B081BF70B083E0916800F0916900B08150
:10151400BA70B01519F4BCE03B2F1CC0B9E03B2FE6
:1015240019C0E0916800F0916900B081BF70B08388
:10153400E0916800F0916900B081FB2FF03019F060
:10154400FA3021F005C0B1E13B2F04C0302D02C0B8
:10155400B9E03B2FB32FD990E990F99009911991F3
:101564002991399108953A932A93402D702D602D35
:10157400502D702DFD01E70FF01D60816F70FD018E
:10158400E70FF01D508152955F70362F262F20955E
:10159400220F220F220F220F322BFC01E70FF01D26
:1015A400E70FF01D3183352F252F2095220F220FB1
:1015B400220F220F322BFC01E70FF01DE70FF01D65
:1015C40030837F5F7630B0F2B02D29913991089540
:1015D4003A932A931A930A93FA92EA92DA92CA9263
:1015E4001B2FF92E0A2FD72EE82EC62E302D202D94
:1015F4008AE6902DA02DB02DF5D114D30092A80128
:101604000092A9010092B4010092AA010092AB01D8
:101614000092AC010092AD010092AE010092AF01C4
:10162400E0EBF1E000820182028203820092B501C4
:101634000092B6010092B7010092B8010092B9017C
:10164400A0916600B09167009E2D8D2D6CE0702DE9
:101654000E945217ACE0BB27A093AC01B093AD013C
:10166400B9E190916600A091670070916800809143
:10167400690058EA61E00E94FF003B2FB01531F485
:10168400B12FA02F9F2D8C2DB6D03B2FB32FC990F7
:10169400D990E990F9900991199129913991089576
:1016A4003A932A931A930A93FA92EA92DA922C972B
:1016B4000B2FFA2ED82EE92E302DB8E1FB9ED00147
:1016C4000024A058BF4F1A2F2B2F013611F4145F9A
:1016D4002F4FBE2DAD2DCE0146DF3B2FB01539F473
:1016E400B22FA12F9CE07C2F8D2F3CD13B2FB32F09
:1016F4002C96D990E990F9900991199129913991F1
:1017040008953A932A931A930A93FA92EA92DA92F0
:10171400CA9222970B2FE92EFA2ED82EC72E302DDF
:10172400B8E1DB9ED0010024A058BF4FA883B98341
:10173400DE011A2F2B2F8AE6902DA02DB02D52D129
:10174400013629F4A881B9811C96A883B9836AD289
:101754000092A8010092A9010092B4010092AA018A
:101764000092AB010092AC010092AD010092AE0177
:101774000092AF01E0EBF1E0008201820282038279
:101784000092B5010092B6010092B7010092B8012F
:101794000092B901A0916600B0916700922F812F49
:1017A40062E0702D0E945217A2E0BB27A093AC0107
:1017B400B093AD01BBE090916600A0916700709179
:1017C40068008091690058EA61E00E94FF003B2FA5
:1017D400B01531F4B02FAF2D9E2D8C2D0CD03B2F96
:1017E400B32F2296C990D990E990F9900991199153
:1017F4002991399108953A932A931A930A93FA9264
:10180400EA921B2FF92E0A2FE82E302D202DB2E25A
:10181400A7E00E94D30086E9902DA02DB02DE2D040
:10182400E0916600F09167001083E0916600F0910A
:101834006700E182A0916600B09167001296902F34
:101844008F2D64E0702D0E9452170092A80100921F
:10185400A9010092B4010092AA010092AB01009286
:10186400AC010092AD010092AE010092AF01E0EB39
:10187400F1E000820182028203820092B5010092AB
:10188400B6010092B7010092B8010092B901A6E036
:10189400BB27A093AC01B093AD01BCE0909166006E
:1018A400A0916700709168008091690058EA61E036
:1018B4000E94FF003B2FB01509F04CC0B5E00E9418
:1018C400E900B770B01519F0BDE03B2F43C0B2E298
:1018D400A3E00E94D3000092A8010092A901009203
:1018E400B4010092AA010092AB010092AC010092F3
:1018F400AD010092AE010092AF01E0EBF1E0008295
:101904000182028203820092B5010092B601009224
:10191400B7010092B8010092B9010092AC010092A3
:10192400AD01B4E190916600A091670070916800E8
:101934008091690058EA61E00E94FF003B2FB015D6
:1019440049F4B9E00E94E900B3FF02C0302D02C09F
:10195400B7E03B2FB32FE990F990099119912991A0
:10196400399108953A932A931A930A93FA92EA9230
:10197400DA928D01F92ED72EE82E202D53D1B2E024
:10198400A02F0E94D300B2E0A12F902F9A2FAA2754
:10199400A92F0E94D300302D09C0B2E0FE2DED2DF9
:1019A400E30FF01DA0810E94D3003F5F3F15A8F311
:1019B400B1E0A1E00E94D300B5E00E94E900B07458
:1019C400B093BD01B015C1F3B1E0A02D0E94D300C6
:1019D400202DB22FD990E990F9900991199129916C
:1019E400399108953A932A931A930A93FA92EA92B0
:1019F400DA92CA92BA92B82EC92EDA2EEB2EB7E03A
:101A0400FB2E3E2D2D2D1C2D0B2D06C0FFEFFF1A96
:101A140036952795179507950015F1E01F072005C2
:101A24003005A0F7F6E1FF1640F0B5E1FB2E8FEF8D
:101A34009927AA27BB278C019D01BAE2AF2D0E94EA
:101A4400D300BCE2A02F0E94D300B02DB990C9905E
:101A5400D990E990F99009911991299139910895B2
:101A64003A932A931A932B2F1A2F302D243010F4E3
:101A7400143018F0B5E23B2F05C020939A00109360
:101A84009B0005D0B32F19912991399108953A9368
:101A9400302DBDE1AEE00E94D300B4E1E0919B00A3
:101AA400FF27EE0FFF1FEE0FFF1FE657FF4FA0812A
:101AB4000E94D300B5E1E0919B00FF27EE0FFF1FCA
:101AC400EE0FFF1FE457FF4FA0810E94D300B9E13E
:101AD400E0919A00FF27EE0FFF1FEE0FFF1FEE0F9E
:101AE400FF1FE659FF4FA0810E94D300BAE1E091A5
:101AF4009A00FF27EE0FFF1FEE0FFF1FEE0FFF1FD1
:101B0400E459FF4FA0810E94D300BCE1E0919A0008
:101B1400FF27EE0FFF1FEE0FFF1FEE0FFF1FE2590F
:101B2400FF4FA0810E94D300BDE1E0919A00FF27FE
:101B3400EE0FFF1FEE0FFF1FEE0FFF1FE059FF4FC9
:101B4400A0810E94D300B32F399108953A93302D88
:101B5400B0919A00B01521F0B0919B00B01521F41A
:101B6400B02DA02D7DDF3B2FB32F399108953A93EB
:101B7400BBE13B2F4DD03B2F301541F40AD03B2F16
:101B8400B01501F484DFA1E0B02D23D0B32F399137
:101B94000895BFE1A02D0E94D300BFE1A0E40E94FC
:101BA400D300B8EC0E941517BFE1A0E452D0BEE107
:101BB400A1E40E94D300BDE2A3E00E94D300B2E1FD
:101BC400AFE30E94D300B3E1AFE30E94D300B02D92
:101BD40008953A932A931A931A2F2B2F302DB1E19B
:101BE400A3E037D01015200531F0B12F0E940A1759
:101BF400B1E1A3E01BD0B32F199129913991089534
:101C0400B1E1A3E026C00895B1E1A2E00FC00895B8
:101C14003A93302D949AB4E60E940A179498B32FFD
:101C240039910895B9E0A1E001C008953A932A9347
:101C34001A932B2F1A2F302DB22F0E94E9003B2F1D
:101C4400B22FA12FA32B0E94D3001991299139916E
:101C540008953A932A931A932B2F1A2F302DB22FCB
:101C64000E94E9003B2FB22FA12FA095A3230E942D
:101C7400D3001991299139910895B9E1A3E70E94FC
:101C8400D300BBE1ADEA0E94D300BCE1AFEF0E94F8
:101C9400D300BDE1AEE10E94D300BEE1A1E00E9409
:101CA400D300BFE1A02D0E94D300B9E0A8E00E94B8
:101CB400D300B4E1A9E10E94D300B5E1A3E10E94FD
:101CC400D300B1E1ABE50E94D300B1E2A6E00E94EB
:101CD400D300BDE2A3E00E94D300B2E2A3E00E94DD
:101CE400D300B3E1AFE30E94D300B02D0895BFEF5A
:101CF400BBBBBFEFBABBBAEBB8BBBAEBB7BBBFEF6A
:101D0400B5BBBFEFB4BBB0E3B2BBBCE3B1BB0E9495
:101D14009516B8EE0E940A17B8EE0E940A170BBE79
:101D240004BEB0EEBBBFBFE0B5BFBBB7BF7BBBBF9C
:101D3400BBB7BF77BBBF5798B9B7BB7FB9BF789460
:101D4400B0E8B8B90E94CA1663DFC49A0E94BF16ED
:101D540094DF0DDFA0E1B02D0E94D816A5EFB0E00E
:101D640091E076E181E00E949200B091F500B09399
:101D74002701B09127010E94E416B9E10E94E9000D
:101D84001B2FB9E10E94E9001B2FBDE1B093EF00C6
:101D9400B4E9B093F000B1E3B093F100BBE0B093C9
:101DA400F200BAE8B093F300BAE8B093F400AFEEEF
:101DB400B0E083EE90E0D7DBA5EFB0E08CE990E0F3
:101DC4000E947017A5EFB0E0C4D7C19A579AB9B76B
:101DD400BB7FB9BF00922F0113DFB6D7B1E0B09338
:101DE4002B0112DF00D4B93911F0B02D01C0B1E0DC
:101DF4002B2FB01531F1A8D7BBEF0E940217B1E029
:101E0400FFD7B091C201FCD7B091C101F9D7B0910D
:101E1400C001F6D7B091BF01F3D7B091C101A09131
:101E2400C201F1E0AF27BA27A091C001BA27A0915F
:101E3400BF01BA27B0932C01B0912C01E1D7BCEFBC
:101E4400DFD7B0912B01B01569F6B0912F01B130F5
:101E540009F043C000922C0100922F01C4D3B93978
:101E640011F0B02D01C0B1E02B2FB01529F1BBEF5B
:101E7400C7D7B1E0C5D7B091C201C2D7B091C101F3
:101E8400BFD7B091C001BCD7B091BF01B9D7B09151
:101E9400C101A091C201F1E0AF27BA27A091C0010E
:101EA400BA27A091BF01BA27B0932C01B0912C019D
:101EB400A7D7BCEFA5D711C0BBEFA2D7B2E0A0D77C
:101EC400B5EA9ED7B0912C01F2E0BF27F5EABF270F
:101ED400B0932C0195D7BCEF93D7B0912F01B230BA
:101EE40009F060C000922C01B5E0B0932801009283
:101EF4002F0100922501B0912E014FD6B93911F06E
:101F0400B02D01C0B1E02B2FB015D9F1BBEF78D7BC
:101F1400B2E076D7B0912C01F2E0BF27B0932C0148
:101F2400B0912E016DD7B0912C01A0912E01BA274A
:101F3400B0932C01B0912D0163D7B0912C01A091E5
:101F44002D01BA27B0932C01302D11C0E32FFF27A8
:101F5400ED5CFE4FB08154D7B0912C01E32FFF27E5
:101F6400ED5CFE4FA081BA27B0932C013F5FB09186
:101F74002D013B1758F3B0912C0142D7BCEF40D749
:101F840011C0BBEF3DD7B2E03BD7B5EA39D7B0912A
:101F94002C01F2E0BF27F5EABF27B0932C0130D71C
:101FA400BCEF2ED7B0912F01B330A1F500922C01D4
:101FB40000922F0100922501B0912E017DD4B939F0
:101FC40011F0B02D01C0B1E02B2FB01591F0BBEF93
:101FD40017D7B4E015D7B9E913D7B0912C01F4E0C1
:101FE400BF27F9E9BF27B0932C010AD7BCEF08D764
:101FF40011C0BBEF05D7B4E003D7B5EA01D7B09160
:102004002C01F4E0BF27F5EABF27B0932C01F8D6E2
:10201400BCEFF6D6B0912F01B63009F06EC0009235
:102024002C0100922F01302DB0913301E32FFF27B3
:10203400EB50FF4FB0833F5F3033B0F3B0912E01CC
:10204400BF3F69F5302DB32F37D42B2F3F5F30318D
:10205400D0F3293991F4BBEFD3D6B6E0D1D6B9E9A0
:10206400CFD6B0912C01F6E0BF27F9E9BF27B09392
:102074002C01C6D6BCEFC4D640C0BBEFC1D6B6E077
:10208400BFD6B5EABDD6B0912C01F6E0BF27F5EA7C
:10209400BF27B0932C01B4D6BCEFB2D62EC0B091FA
:1020A4002E010AD4B93911F0B02D01C0B1E02B2FA3
:1020B400B01591F0BBEFA4D6B6E0A2D6B9E9A0D68C
:1020C400B0912C01F6E0BF27F9E9BF27B0932C01AA
:1020D40097D6BCEF95D611C0BBEF92D6B6E090D69A
:1020E400B5EA8ED6B0912C01F6E0BF27F5EABF27FA
:1020F400B0932C0185D6BCEF83D6B0912F01B430B8
:1021040009F065C000922C0100922F01B0912901C1
:10211400B03661F5B0E6A0912E0183E391E0C0DA18
:10212400B01591F4BBEF6CD6B4E06AD6B9E968D6C1
:10213400B0912C01F4E0BF27F9E9BF27B0932C013B
:102144005FD6BCEF5DD643C0BBEF5AD6B4E058D6D9
:10215400B7EA56D6B0912C01F4E0BF27F7EABF27BF
:10216400B0932C014DD6BCEF4BD631C0B1E6B09341
:102174002901B01561F1B1E6A0912E0183E391E04C
:102184008FDAB01599F4BBEF3BD6B4E039D6B9E990
:1021940037D6B0912C01F4E0BF27F9E9BF27B093FB
:1021A4002C012ED6BCEF2CD6CFD511C0BBEF28D630
:1021B400B4E026D6B7EA24D6B0912C01F4E0BF27C8
:1021C400F7EABF27B0932C011BD6BCEF19D6B09108
:1021D4002F01B53009F039CE00922C0100922F0165
:1021E400B0912E0195EFA0E07DED80E057ED60E029
:1021F40069D42B2F293991F4BBEF02D6BAE300D668
:10220400B9E9FED5B0912C01F5E0BF27F9E9BF2764
:10221400B0932C01F5D5BCEFF3D517CEBBEFF0D5B9
:10222400BAE3EED5B7EAECD5B0912C01F5E0BF27BF
:10223400F7EABF27B0932C01E3D5BCEFE1D505CE77
:102244000895FA93EA93BA93AA939A938A937A9302
:102254006A935A934A933A931A920A921FB61A921D
:10226400002400922F01D0D5BB3F11F0B02D01C046
:10227400B1E0B0933201B01509F4A5C1C5D5B0934E
:102284003001B0913001B015E9F4BED5BC3F11F076
:10229400B02D01C0B1E0B0933101B01551F043D578
:1022A40000922B01BBEFACD5B1E0AAD5BCEFA8D509
:1022B40009C000922E0100922D01BFEFB0933001AE
:1022C40000922F01B0913001B13081F49DD5B093CB
:1022D4002C019AD5BC3F11F0B02D01C0B1E0B093F0
:1022E4003101B01519F0B1E0B0932F01B091300174
:1022F400B23001F589D5B0932E0186D5B0932D0166
:1023040083D5B0932C0180D5BC3F11F0B02D01C012
:10231400B1E0B0933101B01521F0B2E0B0932F01D8
:1023240009C000922E0100922D01BFEFB09330013D
:1023340000922F01B0913001B430B1F565D5B0935E
:102344002E0162D5B0932D01302DE32FFF27ED5CD4
:10235400FE4F00823F5F3033C0F3302D07C054D5A9
:10236400E32FFF27ED5CFE4FB0833F5FB0912D015B
:102374003B17A8F349D5B0932C0146D5BC3F11F0C7
:10238400B02D01C0B1E0B0933101B01521F0B3E03C
:10239400B0932F0109C000922E0100922D01BFEFCE
:1023A400B093300100922F01B0913001B134F9F4AF
:1023B4002BD5B0932E0128D5B093330125D5B093F6
:1023C4002C0122D5BC3F11F0B02D01C0B1E0B09377
:1023D4003101B01521F0B6E0B0932F0108C0BFEF72
:1023E400B0932E01BFEFB093300100922F01B09152
:1023F4003001BA3091F508D5B0932E0105D5B093CC
:102404002D01302D07C000D5E32FFF27ED5CFE4FD3
:10241400B0833F5FB0912D013B17A8F3F5D4B0937F
:102424002901F2D4B0932C01EFD4BC3F11F0B02DAC
:1024340001C0B1E0B0933101B01521F0B4E0B09324
:102444002F010BC00092290100922E0100922D0150
:10245400BFEFB093300100922F01B0913001BA3137
:1024640009F045C0D1D4B0932701CED4B0932C0148
:10247400CBD4BC3F11F0B02D01C0B1E0B093310119
:10248400B01561F150D4B0912701B093F500A5EFD8
:10249400B0E091E076E181E00E947D00BBEFB0D432
:1024A400BAE1AED4B0912701ABD4B0912701FAE1DF
:1024B400BF27A6D4BCEFA4D4A5EFB0E091E076E1A9
:1024C40081E00E949200B091F500B0932701A0E151
:1024D400B02D6CD4B091270175D409C000922E019F
:1024E40000922D01BFEFB093300100922F01B09103
:1024F4003001BA3249F588D4B093260185D4B0931B
:102504002C0182D4BC3F11F0B02D01C0B1E0B093D6
:102514003101B01581F0B09126010AD4BBEF70D41B
:10252400BAE26ED4B09126016BD4B0912C0168D478
:10253400BCEF66D409C000922E0100922D01BFEFBA
:10254400B093300100922F01B0913001BA33D9F524
:102554005BD4B0932E01302D57D4E32FFF27EB50DB
:10256400FF4FB0833F5F3630B8F3302D4DD4E32FA7
:10257400FF27E352FF4FB0833F5F3630B8F3302D6F
:1025840043D4E32FFF27E952FF4FB0833F5F363038
:10259400B8F33AD4B0932C0137D4BC3F11F0B02D2A
:1025A40001C0B1E0B0933101B01521F0B5E0B093B2
:1025B4002F0109C000922E0100922D01BFEFB093AC
:1025C400300100922F0119901FBE09901990399182
:1025D400499159916991799189919991A991B99167
:1025E400E991F99118953A93BAE03B2FB0E14CD3B5
:1025F4000BDBB2E59BEBA1E00E948804B093BA0127
:10260400B091BA01B01511F4302D01C0315030151C
:1026140081F7B091BA01B015E9F4B02D9FEBA1E0B8
:102624000E942E05B093BA01B091BA01B015B1F46D
:10263400AFEBB1E08EEB91E00E942607B093BA01B4
:10264400B091BA01B01551F4DBDAB9E9B093BA012B
:1026540005C004C0D5DAB5EAB093BA01399108953A
:102664003A932A932B2F00922A01B22F95EFA0E0E0
:102674000E94E807B093BA01B091BA01B015C1F451
:10268400302DE32FFF27EB50FF4FB081E091250160
:10269400FF27ED5CFE4FB083B0912501BF5FB0937F
:1026A40025013F5F303168F3B9E9B093BA0107C03F
:1026B400B0912A01B015C9F6B5EAB093BA012991CF
:1026C400399108953A932A932B2F00922A01B22F1D
:1026D40095EFA0E00E94E807B093BA01B091BA0167
:1026E400B015C1F4302DE32FFF27EB50FF4FB0811D
:1026F400E0912501FF27ED5CFE4FB083B0912501E9
:10270400BF5FB09325013F5F303168F3B9E9B093FF
:10271400BA0107C0B0912A01B015C9F6B5EAB09361
:10272400BA012991399108953A932A932B2F009253
:102734002A01B22F95EFA0E00E94E807B093BA01F6
:10274400B091BA01B015C1F4302DE32FFF27EB503F
:10275400FF4FB081E0912501FF27ED5CFE4FB08370
:10276400B0912501BF5FB09325013F5F303168F31D
:10277400B9E9B093BA0107C0B0912A01B015C9F6FE
:10278400B5EAB093BA012991399108953A932A93FD
:102794002B2F00922A01302DE0912501FF27ED5CBB
:1027A400FE4FB081E32FFF27EB50FF4FB083B09172
:1027B4002501BF5FB09325013F5F303168F3B22F2D
:1027C40095EFA0E00E942B09B093BA01B091BA0131
:1027D400B01521F4B9E9B093BA0107C0B0912A0148
:1027E400B01569F7B5EAB093BA0129913991089502
:1027F4003A932A932B2F00922A01302DE091250140
:10280400FF27ED5CFE4FB081E32FFF27EB50FF4F16
:10281400B083B0912501BF5FB09325013F5F303194
:1028240068F3B22F95EFA0E00E942B09B093BA0190
:10283400B091BA01B01521F4B9E9B093BA0107C057
:10284400B0912A01B01569F7B5EAB093BA0129919C
:10285400399108953A932A932B2F00922A01302D0F
:10286400E0912501FF27ED5CFE4FB081E32FFF27A8
:10287400EB50FF4FB083B0912501BF5FB0932501AA
:102884003F5F303168F3B22F95EFA0E00E942B092F
:10289400B093BA01B091BA01B01521F4B9E9B0937B
:1028A400BA0107C0B0912A01B01569F7B5EAB0932F
:1028B400BA012991399108953A932A931A930A9364
:1028C4000B2FB02FBB0FBB0F2B2FB4E61B2F9CD9A4
:1028D400B6E29BEBA1E00E9488043B2F301511F473
:1028E400102D01C01150101599F7301509F070C062
:1028F400B02D9FEBA1E00E942E05B01511F0B02D74
:1029040001C0B1E03B2FB01509F465C0AFEBB1E0F5
:102914008EEB91E00E942607B01511F0B02D01C096
:10292400B1E03B2FB01509F456C0B1E69FEBA1E02E
:10293400802F722F7D5F0E94830BB01511F0B02D94
:1029440001C0B1E03B2FB01509F445C0001529F1D1
:10295400B22F1CDFB93911F0B02D01C0B1E03B2F0B
:10296400B015C9F1B22FBF5F43DFB93911F0B02DF3
:1029740001C0B1E03B2FB01571F1B22FBE5F6ADF29
:10298400B93911F0B02D01C0B1E03B2FB01519F1E8
:1029940037D9B9E93B2F1FC01EC0B22FBF5F28DF54
:1029A400B93911F0B02D01C0B1E03B2FB01599F049
:1029B400B22FBE5F4FDFB93911F0B02D01C0B1E0C5
:1029C4003B2FB01541F01CD9B9E93B2F04C003C01B
:1029D40017D9B5EA3B2F0991199129913991089595
:1029E4003A932A931A930A93FA921B2FF92E0A2FD9
:1029F400B12FBB0FBB0F2B2FB4E63B2F05D9B2E58C
:102A04009BEBA1E00E948804B093BA01B091BA0193
:102A1400B01511F4302D01C03150301581F7B0914B
:102A2400BA01B01509F044C0B02D9FEBA1E00E949B
:102A34002E05B01511F0B02D01C0B1E0B093BA016C
:102A4400B015D1F1AFEBB1E08EEB91E00E94260717
:102A5400B01511F0B02D01C0B1E0B093BA01B015BA
:102A640059F1B1E69FEBA1E073EE80E0622F6D5F58
:102A74000E94EA0AB01511F0B02D01C0B1E0B09384
:102A8400BA01B015C9F0B22FBD5FA02F9F2D0E94CF
:102A94002B09B01511F0B02D01C0B1E0B093BA010B
:102AA400B01551F0ADD8B9E9B093BA0105C004C06E
:102AB400A7D8B5EAB093BA01F9900991199129916F
:102AC400399108953A932A931A930A93FA92EA92BF
:102AD400DA92CA92BA9260971B2FF92E0A2FD72E38
:102AE400E82EB52EC62EB02FAF2D83EE90E00E94B7
:102AF400B50A302DFE2DED2DE30FF01DB081FE0142
:102B0400E30FF01DB0833F5F3630A0F3B8E0FE0161
:102B1400A32F3F5FEA0FF01DB083B7E7FE01A32F99
:102B24003F5FEA0FF01DB083BFE8FE01A32F3F5FB4
:102B3400EA0FF01DB083FE01B32F3F5FEB0FF01DD2
:102B44000082232F302DFC2DEB2DE30FF01DB081DF
:102B5400FE01E20FF01DB0832F5F3F5F363098F324
:102B6400B12F9C2FAD2F3CDFB093BA01B091BA01C5
:102B7400B93929F4B9E9B093BA0104C003C0B7EA7A
:102B8400B093BA016096B990C990D990E990F99040
:102B9400099119912991399108953A932A931A9395
:102BA4000A930B2FB02FBB0FBB0F2B2FB4E61B2F99
:102BB4002BD8B2E59BEBA1E00E9488043B2F301593
:102BC40011F4102D01C01150101599F7301509F0AA
:102BD40052C0B02D9FEBA1E00E942E05B01511F05C
:102BE400B02D01C0B1E03B2FB01509F448C0AFEBE4
:102BF400B1E08EEB91E00E942607B01511F0B02DE4
:102C040001C0B1E03B2FB015D1F1B0E69FEBA1E0DC
:102C1400802F722F7D5F0E94830BB01511F0B02DB1
:102C240001C0B1E03B2FB01551F1B22F19DDB93914
:102C340011F0B02D01C0B1E03B2FB01501F1B22F5E
:102C4400BF5F40DDB93911F0B02D01C0B1E03B2FB9
:102C5400B015A9F0B22FBE5F67DDB93911F0B02D00
:102C640001C0B1E03B2FB01551F00E94020EB9E94A
:102C74003B2F05C004C00E94020EB5EA3B2F099108
:102C84001991299139910895A02D07C09FEFEA2F3A
:102C9400FF27EB50FF4F9083AF5FAB17B8F3089556
:102CA400FA93EA93BA93AA939A938A937A936A9338
:102CB4005A934A931A920A921FB61A920024A7EFC3
:102CC400B2ECBDBDACBDB0912801B150B0932801A8
:102CD40029D0B0912801B01511F400922A0119905D
:102CE4001FBE0990199049915991699179918991DF
:102CF4009991A991B991E991F99118951A920A9229
:102D04001FB61A92002419901FBE099019901895A5
:102D14001A920A921FB61A92002419901FBE0990A3
:102D2400199018950895C198B4E672D0C19A08957F
:102D34003A933B2FC198BAE03B9FD0010024BA2FAD
:102D440067D0C19A39910895C198B8EE61D0C19AFB
:102D540008953A932A93A5EFB0E0C8D02A2F302DD6
:102D640007C0E32FFF27EB50FF4FB08149D03F5FEF
:102D74003217B8F32991399108950FBCB5E0BEBD5F
:102D8400A8E1BEEFBDBDACBD08BEB4E0B9BF0895B7
:102D9400B8B3B06BB8BBB7B3B06AB7BBBDB1B365BA
:102DA400BDB90895BFB9779BFECF0895CD01892F92
:102DB400992780BDA9B992E09BB998E99AB996E898
:102DC40090BD0895FB2FF03049F0F13051F0F2300E
:102DD40059F0F33061F0F43069F00FC0AFECA9B9E9
:102DE4000895A7E6A9B90895A4E4A9B90895A3E3A9
:102DF400A9B90895A2E2A9B90895A3E3A9B90895C8
:102E04005D9BFECFBCB908955F9BFECFBCB1089516
:102E1400EFE9FFE0E150F040E9F700C00000B150F5
:102E2400B015B1F7089500C0B150B015E1F7089599
:102E3400EB2FE92799231CF4909581959F4FBB2391
:102E44001CF4B095A195BF4F18D0EE231CF4B09597
:102E5400A195BF4F0895EB2F99231CF4909581956C
:102E64009F4FBB231CF4B095A195BF4F16D0EE2302
:102E74001CF4B095A195BF4F089577276627F0E11C
:102E8400AA0FBB1F661F771F6817790718F0681B06
:102E9400790BA395FA95A1F70895EFDFDB01089567
:102EA400FC01CB01BD0110C011901D9211901D9227
:102EB40011901D9211901D9211901D9211901D92CE
:102EC40011901D9211901D92089770F7089621F0A9
:102ED40011901D920197E1F7DB010895FC01CD01EA
:102EE40071917D937723E1F7DC010895FD019D91B4
:0C2EF4009923E9F7AE1BBF0B119708955E
:1000000062C0FFFF0C9480160C948A16D7C2FFFFC3
:10001000FFFFFFFFFFFFFFFFFFFFFFFFFFFFFFFFF0
:10002000FFFFFFFF0C945216FFFFFFFFFFFFFFFFD4
:08003000FFFFFFFF0C942311F8
:00000001FF
